:100000000C9446000C9463000C9463000C94630001
:100010000C9463000C9463000C9463000C946300D4
:100020000C9463000C9463000C9463000C946300C4
:100030000C9463000C9463000C9463000C947700A0
:100040000C9463000C9463000C9463000C946300A4
:100050000C9463000C9463000C9463000C94630094
:100060000C9463000C9463000C9463000C94630084
:100070000C9463000C9463000C9463000C94630074
:100080000C9463000C9463000C94630011241FBE55
:10009000CFEFD0E1DEBFCDBF11E0A0E0B1E0E4EBF7
:1000A000F1E100E00BBF02C007900D92A639B10745
:1000B000D9F712E0A6E9B1E001C01D92A939B10754
:1000C000E1F70C94BD000C940000F8948FEF8ABB0C
:1000D0008BBB84BB15BA80B7886080BF8FE183BFBC
:1000E00082E081BF87B7826087BF789408951F92AE
:1000F0000F920FB60F9211242F933F934F935F935C
:100100006F937F938F939F93AF93BF93EF93FF93DF
:100110000E942902FF91EF91BF91AF919F918F9122
:100120007F916F915F914F913F912F910F900FBEF3
:100130000F901F901895CF930E9465000E94C701F1
:10014000C0E0609198026623E1F7C930D0F781E002
:1001500090E00C2E02C0880F991F0A94E2F74FEF2F
:100160000E9455028C2F0E94710160E070E08AE7C6
:1001700094E40E941B01CF5FE4CFCFEFD0E1DEBF5C
:10018000CDBF0E949B0080E090E00C94D9089F9224
:10019000AF92BF92CF92DF92EF92FF920F931F9395
:1001A000CF935B016C0120E030E040E452E40E9418
:1001B0002905DC01CB01BC01CD010E945A02DC0102
:1001C000CB01982EC0E0C81758F52BEA3AEA4AEA64
:1001D00050E4C601B5010E940E047B018C0120E0B1
:1001E00030E040E85FE30E944506882314F481E094
:1001F00012C020E030E04FE753E4C801B7010E948D
:10020000D905181614F480E006C0C801B7010E9491
:100210005A02DC01CB018A95F1F7CF5FC915A8F22C
:10022000CF911F910F91FF90EF90DF90CF90BF90F3
:10023000AF909F9008959F92AF92BF92CF92DF921E
:10024000EF92FF920F931F93CF935B016C0120E01D
:1002500030E040E85DE30E940E04DC01CB01BC010C
:10026000CD010E945A02DC01CB01982EC0E0C817D4
:1002700068F520E030E04AE755E4C601B5010E9488
:100280000E047B018C0120E030E040E85FE30E9437
:10029000450688231CF481E090E013C020E03FEF86
:1002A0004FE757E4C801B7010E94D90518161CF49E
:1002B00080E090E006C0C801B7010E945A02DC014C
:1002C000CB010197F1F7CF5FC91598F2CF911F913C
:1002D0000F91FF90EF90DF90CF90BF90AF909F90E5
:1002E0000895CF93DF93CDB7DEB7C356D0400FB696
:1002F000F894DEBF0FBECDBF282FAE014F5F5F4F1A
:10030000DA01E0E0F1E093E601900D929150E1F71F
:100310008BE0809396029093970290919702809140
:100320009602981728F533278BE090E0289FB001BC
:10033000299F700D389F700D11249B0180919702A9
:10034000A82FBB27A956BE4F80919702F901E80F4D
:10035000F11DE40FF51F80818C93809197028F5FD0
:10036000809397029091970280919602981730F3AC
:10037000109296018FEF80939802CD59DF4F0FB600
:10038000F894DEBF0FBECDBFDF91CF91089589E114
:100390008093960210929702909197028091960214
:1003A000981780F480919702E82FFF27E956FE4FB7
:1003B000809197028F5F8083809197028F5F8093F7
:1003C0009702EACF109296018FEF809398020895DA
:1003D000CF93DF93CDB7DEB7AB970FB6F894DEBF00
:1003E0000FBECDBF9E012F5F3F4FD901E3E6F1E085
:1003F0009BE201900D929150E1F78BE2809396027F
:10040000909397029091970280919602981798F492
:1004100080919702A82FBB27A956BE4F80919702C3
:10042000F901E80FF11D80818C93809197028F5F15
:1004300080939702E7CF109296018FEF80939802F6
:10044000AB960FB6F894DEBF0FBECDBFDF91CF9154
:100450000895809198028F3F39F580919601E82F99
:10046000FF27E956FE4FE081809196018F5F8093D0
:100470009601EE23B1F080E0EF3F09F08CE185BDFD
:10048000E3BD85B38093970285B3807F8093970205
:1004900080919702825F809397028091970285BB3B
:1004A0000895E5BDE093980208954F3F11F4481B6D
:1004B0004BBB0895EF92FF920F931F937B018C012A
:1004C00020E030E040E05FE40E940F0688239CF0CB
:1004D00020E030E040E05FECC801B7010E94A803D3
:1004E000DC01CB01BC01CD010E947B066050704055
:1004F0008040904804C0C801B7010E947B061F914C
:100500000F91FF90EF900895A0E0B0E0EAE8F2E0EC
:100510000C94A2088C017B015A01DC018C91823081
:1005200058F0FB019081923010F4A7010BC1843088
:1005300029F4943009F4A6C0A80104C19430A9F3A9
:10054000923009F4A9C0823081F3F801C280D380CF
:10055000FB0162817381F8012481358146815781D5
:10056000F7016480758086809780C601861B970B93
:1005700097FDD8C080970CF46CC06C157D050CF00D
:10058000ADC0662477244301F8016181F7018181C0
:10059000681709F499C0662309F491C0621A730AB6
:1005A000840A950AA401930157FDC0C0F501118288
:1005B000B60119012A0179018A0139014A01089419
:1005C0006108710881089108FFEF6F16FFEF7F0641
:1005D000FFEF8F06FFE39F06F0F4A8019701220FBB
:1005E000331F441F551F19012A01B6016150704085
:1005F0006B0179018A0139014A0108946108710887
:10060000810891088FEF68168FEF78068FEF8806C4
:100610008FE3980610F383E0D5018C9357FC64C0F8
:10062000F501248335834683578373836283A50151
:1006300089C06F5F7F4FD401C30181709070A0703B
:10064000B0709694879477946794682A792A8A2A56
:100650009B2A6C157D056CF311C00894C11CD11C3C
:10066000DA01C90181709070A070B07056954795FD
:1006700037952795282B392B4A2B5B2BC616D70687
:1006800064F382CFF8019181FB018181981709F40D
:1006900053CF4EE851E056C0823009F04DCFDA0119
:1006A000F80188E001900D928150E1F7F801818115
:1006B000F70191818923F5018183A50143C02619A2
:1006C00037094809590970CFF5016183B601260D34
:1006D000371D481D591D19012A019DCF6B0120E0CE
:1006E00030E040E050E050CFD201C101B695A7956F
:1006F0009795879521E030E040E050E022223322B8
:1007000044225522282A392A4A2A5B2AF5012482C2
:100710003582468257820894C11CD11CD382C28282
:10072000A50110C0909581959F4F24CF81E0F501E0
:100730008183B60150954095309521953F4F4F4F9D
:100740005F4F37CFCA01E2E1CDB7DEB70C94BE08E8
:10075000A0E2B0E0EEEAF3E00C94B008DC01CB01DB
:10076000898F9A8FAB8FBC8F2D8F3E8F4F8F58A361
:10077000BE016F5F7F4FCE0149960E94B5078E0183
:10078000075F1F4FB801CE014D960E94B507AE011D
:100790004F5E5F4FB801CE0101960E9484020E9415
:1007A000CD06DC01CB01BC01CD01E4E0A0960C94A8
:1007B000CC08A0E2B0E0EFEDF3E00C94B008DC016F
:1007C000CB01898F9A8FAB8FBC8F2D8F3E8F4F8F30
:1007D00058A3BE016F5F7F4FCE0149960E94B507B7
:1007E0008E01075F1F4FB801CE014D960E94B507DD
:1007F0008A8591E089278A87AE014F5E5F4FB801F5
:10080000CE0101960E9484020E94CD06DC01CB013C
:10081000BC01CD01E4E0A0960C94CC08A0E2B0E0CD
:10082000E4E1F4E00C94A208DC01CB01898F9A8FFB
:10083000AB8FBC8F2D8F3E8F4F8F58A3BE016F5F44
:100840007F4FCE0149960E94B50769E070E06C0FBA
:100850007D1FCE014D960E94B507FE01319666249C
:1008600077244301130124018981823098F099850E
:10087000923058F420E091818A85981321E02A87EC
:1008800069E070E06C0F7D1FD9C0843059F492305C
:1008900009F45BC020E091818A85981321E02183CF
:1008A000BF01CCC0943009F44DC0823099F392302E
:1008B00009F3ED80FE800F8118852D853E854F85DB
:1008C0005889640153016FE170E00CC0220F331F9F
:1008D000441F551F16950795F794E7946150704093
:1008E00077FD36C0D801C70181709070A070B070DC
:1008F000892BC9F080E090E0220E331E441E551E65
:10090000221633064406550610F481E090E0AA272B
:1009100097FDA095BA2F8A0D9B1DAC1DBD1D680EBD
:10092000791E8A1E9B1EAA0CBB1CCC1CDD1C57FF0B
:10093000CDCF81E090E0A0E0B0E0A82AB92ACA2A91
:10094000DB2AC4CF823009F095CF6EE871E076C023
:10095000228133818B859C85280F391F2E5F3F4F65
:10096000A90160E091818A85981361E06A8B97FE06
:100970000FC02FC0CA010197AC019C01660C771C07
:10098000881C991C57FC41C0220C331C441C551C6C
:1009900090E0691690E0790690E0890690E4990667
:1009A00048F33C8B2B8BD401C3018F779070A070E0
:1009B000B07080349105A105B10581F16D8A7E8A00
:1009C0008F8A988E83E0898B61E170E06C0F7D1FC8
:1009D00035C02F5F3F4FA901D401C30181709070D2
:1009E000A070B070892B61F0569447943794279487
:1009F00080E090E0A0E0B0E8282A392A4A2A5B2A61
:100A00009694879477946794C3CF81E090E0A0E0B8
:100A1000B0E0682A792A8A2A9B2AB6CF67FC05C0EB
:100A2000211431044104510449F280E490E0A0E033
:100A3000B0E0680E791E8A1E9B1EC0CFCB010E94BB
:100A4000CD06DC01CB01BC01CD01E2E1A0960C9406
:100A5000BE08A8E1B0E0EFE2F5E00C94AA08DC01E2
:100A6000CB01898B9A8BAB8BBC8B2D8B3E8B4F8BA9
:100A7000588FBE016F5F7F4FCE0141960E94B50730
:100A80008E01075F1F4FB801CE0145960E94B50742
:100A9000FE0131962981223008F45FC03985323059
:100AA00010F4B8017BC081819A8589278183243025
:100AB00009F455C0223009F452C0343009F454C04E
:100AC000323009F458C06B817C818B859C85681B12
:100AD000790B2D813E814F815885ED84FE840F85F1
:100AE00018892E153F054007510730F4220F331F98
:100AF000441F551F615070407C836B8380E090E001
:100B0000A0E0B0E4AA24BB2465012E153F054007F0
:100B1000510740F0A82AB92ACA2ADB2A2E193F0910
:100B2000400B510BB695A79597958795220F331FCC
:100B3000441F551F0097A105B10539F7D601C5011E
:100B40008F779070A070B07080349105A105B105C9
:100B5000A9F0A482B582C682D782BF011FC0231725
:100B6000E1F76EE871E01AC01D821E821F821886AE
:100B70001C821B82F2CF84E08983EFCFA7FC05C0E3
:100B8000211531054105510521F380E490E0A0E0F5
:100B9000B0E0A80EB91ECA1EDB1EDBCFCB010E943F
:100BA000CD06DC01CB01BC01CD01EAE068960C94D6
:100BB000C608A8E1B0E0EFEDF5E00C94B008DC0168
:100BC000CB01898B9A8BAB8BBC8B2D8B3E8B4F8B48
:100BD000588FBE016F5F7F4FCE0141960E94B507CF
:100BE0008E01075F1F4FB801CE0145960E94B507E1
:100BF0008981823018F08985823018F42FEF3FEF19
:100C000009C0B801CE0101960E942F08282F332772
:100C100027FD3095C901E4E068960C94CC08A8E162
:100C2000B0E0E5E1F6E00C94B008DC01CB01898B83
:100C30009A8BAB8BBC8B2D8B3E8B4F8B588FBE0111
:100C40006F5F7F4FCE0141960E94B5078E01075F0F
:100C50001F4FB801CE0145960E94B50789818230A9
:100C600018F08985823018F42FEF3FEF09C0B801E2
:100C7000CE0101960E942F08282F332727FD30959B
:100C8000C901E4E068960C94CC08A8E1B0E0EBE47C
:100C9000F6E00C94B008DC01CB01898B9A8BAB8B0E
:100CA000BC8B2D8B3E8B4F8B588FBE016F5F7F4F60
:100CB000CE0141960E94B5078E01075F1F4FB80114
:100CC000CE0145960E94B5078981823018F089854A
:100CD000823018F421E030E009C0B801CE0101965D
:100CE0000E942F08282F332727FD3095C901E4E003
:100CF00068960C94CC08ACE0B0E0E1E8F6E00C9427
:100D0000B208DC01CB0189879A87AB87BC87BE011B
:100D10006F5F7F4FCE0109960E94B50789818230AF
:100D200011F0823028F460E070E080E090E031C0A3
:100D3000843039F02B813C8137FDF5CF2F313105DF
:100D40006CF08A81882329F060E070E080E090E810
:100D500020C06FEF7FEF8FEF9FE71BC08EE190E029
:100D6000821B930B2D813E814F81588504C056957F
:100D70004795379527958A95D2F78A81882339F048
:100D800050954095309521953F4F4F4F5F4FCA0189
:100D9000B901E2E02C960C94CE08A0E0B0E0E3EDBF
:100DA000F6E00C94A808882499245401DC01FC0185
:100DB00024813581468157818181082F112760E088
:100DC00070E08C91823020F46FEF70E04061A4C03D
:100DD000843009F464C0823009F463C02115310500
:100DE0004105510509F498C0FD0182819381FFEF0F
:100DF00082389F070CF050C0A2E8EA2EAFEFFA2E1F
:100E0000E81AF90A8AE1E816F1040CF06BC06B01EC
:100E100081E090E0A0E0B0E00E2C04C0880F991FA4
:100E2000AA1FBB1F0A94D2F70197A109B109822317
:100E30009323A423B5230097A105B10519F0F1E090
:100E4000CF2ED12C04C05695479537952795EA9417
:100E5000D2F7C601AA2797FDA095BA2F282B392BC8
:100E60004A2B5B2BDA01C9018F779070A070B070AC
:100E700080349105A105B105D1F1215C3F4F4F4F61
:100E80005F4F2030E0E03E07E0E04E07E0E45E0721
:100E900008F161E070E01EC0803891053CF06FEF12
:100EA00070E020E030E040E050E036C0BC01615826
:100EB0007F4FDA01C9018F779070A070B0708034D5
:100EC0009105A105B105D1F0215C3F4F4F4F5F4F18
:100ED00057FD1BC097E056954795379527959A95EE
:100EE000D1F71AC020E030E040E050E0BBCF27FF50
:100EF000C8CF205C3F4F4F4F5F4FC3CF27FFE8CF96
:100F0000205C3F4F4F4F5F4FE3CF56954795379546
:100F100027956F5F7F4FDECF822E932E942F9F7782
:100F20008A2D8078A82EA92A962F9795992797958C
:100F30008A2D8F77A82EA92A76956795962F9F7769
:100F40008B2D8078B82EB92A902F97959927979551
:100F50008B2D8F77B82EB92AD501C401BC01CD01E4
:100F6000ECE0CDB7DEB70C94C408CF93DF93FC015F
:100F7000DB01408151812281622F6F7770E0221F57
:100F80002227221F9381892F880F822B282F332716
:100F9000991F9927991FED0199832115310541F476
:100FA0004115510561057105E1F482E08C9354C04F
:100FB0002F3F310509F441C02F573040FD013383E5
:100FC000228383E08C9387E0440F551F661F771FB1
:100FD0008A95D1F77064ED014C835D836E837F83C6
:100FE0003BC022E83FEFF901C7E0440F551F661FE1
:100FF000771FCA95D1F783E08C93403080E0580783
:1010000080E0680780E4780778F4440F551F661F76
:10101000771F21503040F9014030C0E05C07C0E04C
:101020006C07C0E47C0788F3ED01FB83EA83FD01D4
:1010300044835583668377830FC04115510561054D
:10104000710519F484E08C9307C064FF03C081E04C
:101050008C93C1CF1C92BFCFDF91CF9108950F9396
:101060001F93CF93DF93FC01DB018081823018F066
:101070009C91923018F461E070E05EC08430C1F061
:10108000843001F1943009F447C0823009F44BC038
:10109000823009F44EC09230A9F04181ED0189817E
:1010A0004817B9F0442389F08FEF9FEFBC0144C08B
:1010B000943031F7EB018981682F77278181681B94
:1010C00071093AC08181882379F781E090E0BC0101
:1010D00033C022813381ED018A819B81821793077E
:1010E0000CF3281739079CF004811581268137817C
:1010F000FD01648175818681978160177107820780
:10110000930780F2061717072807390778F4442356
:1011100059F281E090E0DBCFFD018181882321F24B
:1011200081E090E0D4CF923009F0B2CF60E070E07F
:1011300003C0ED018981F2CFCB01DF91CF911F91E7
:101140000F9108952F923F924F925F926F927F92EC
:101150008F929F92AF92BF92CF92DF92EF92FF92C7
:101160000F931F93CF93DF93CDB7DEB7CA1BDB0B73
:101170000FB6F894DEBF0FBECDBF09942A88398818
:1011800048885F846E847D848C849B84AA84B9841F
:10119000C884DF80EE80FD800C811B81AA81B9812B
:1011A000CE0FD11D0FB6F894DEBF0FBECDBFED013F
:0411B0000895FFCFD0
:1011B400050A0F141919140F0A0500196419641982
:1011C400641964196400050519050519050519193B
:1011D40000C8C8FFC8C8FFC8C8FFFF00C8FFC8FFD1
:1011E400C8FF0000000000F0FFF0FFF0FF00000067
:1011F40000006464FF6464FF6464FF64000DFF1412
:10120400FF0DFF14FF0DFF0001FF02FF03FF04FFAA
:1012140005FF000AFF050A050A050A0DFF0A0D0A63
:101224000D0A0D11FF0D110FFF0C0F0DFF0A0D0C10
:10123400FF11FF1110100D0D0C0C0A0AFF00000025
:06124400000000000000A4
:00000001FF
